:10000000B700000067808000735040307350403468
:1000100081400141814101428142014381430144C8
:100020008144814601478147970100209381817D6A
:10003000F32340F1B70200009382020063F47200E0
:100040006F006018170100201301C17BB702000088
:1000500093820240638603001E837D13E31F03FE29
:1000600033015140330401006F004000411106C6C6
:100070000008137101FF732540F197000000E7802D
:10008000201221C997000000E780401137050020A9
:1000900013050500B7050020938505006377B500BB
:1000A000232005001105E36DB5FE3705002013057B
:1000B0000500B70500009385851F3706002013064D
:1000C00006006378C500944114C111059105E36CE5
:1000D000C5FE97000000E780E00D97000000E78074
:1000E00060080000397106C016C21AC41EC62AC8AC
:1000F0002ECA32CC36CE3AD03ED233050100EF00C4
:100100000002824092422243B2434245D2456246B7
:10011000F2460257925713014102730020300A84BD
:10012000137101FFF325203463C7050022811703F3
:10013000000067006306139515000581B145637CD7
:10014000B5000A05B70500009385851C2E951C4156
:1001500099C3228182872281170300006700E3038D
:1001600037150240C1450CCD3715014093050005F8
:100170000CC1894537460F00130606244CC5B286CC
:1001800099C2FD16FDFE23260500B286E5DAFD16AE
:10019000FDFEEDB701A001A0228182800A841371C7
:1001A00001FF01C573005010F5BF05452281828013
:1001B0000A84137101FF370500001305450E731003
:0801C00055302281828001A06C
:1001C8009601000096010000000000009601000062
:1001D8009601000096010000000000009601000052
:1001E8009601000096010000000000009601000042
:00000001FF
